:020000020000FC
:100000005ECDA4C1000000001FC0000092C000002F
:1000100000009CC000000000000000000203040675
:10002000080C10182030406080000406080C1018DE
:100030002030406080A0C00000070F1F3F00050572
:100040000D050305030302004FB662FD0EC05520E7
:1000500009F00994C52DC095089483FDC795C4BDCA
:10006000C093A10064604FBE1895C09164000894CD
:1000700083FDC795C4BDC093A1006B7FC091640090
:10008000CF3F09F41FC070FF02C082FD05C04FBE04
:10009000C098C198C2981895C098C198C29875FD2B
:1000A0000DC065FD0BC0C9E0CA95F1F7C091B30062
:1000B000C0FD939AC1FD949AC2FD959A2092A10029
:1000C0004FBE189524BCCC27C064C8BF6460F6CF6F
:1000D000C1CF70FFBFCF65FDBDCFC09ABBCF70FF52
:1000E000B9CF65FDB7CFC19AB5CF70FFB3CF65FD6E
:1000F000B1CFC29AAFCF939870FFACCF65FDAACFB6
:10010000C7E0CA95F1F7C09AA5CF949870FFA2CF27
:1001100065FDA0CFC7E0CA95F1F7C19A9BCF95982E
:1001200070FF98CF65FD96CFC7E0CA95F1F7C29AE8
:1001300091CF4FB6C9B7CF7EC9BF6E7FCCB5CE0DBC
:10014000DDB5DF1DDBBDCABD4FBE18953FB68F7E46
:10015000ABB7A074A2118061A0E0ABBFA9B7AE7F1E
:10016000A9BF7894A0916800AA2341F085FD2AC018
:10017000A0916800AA95A093680024C040E050E0D8
:1001800085FD14C0A0B396FDA095A2FD4FEFA3E09E
:1001900096FDA2E0A5BFAA27A064AABF8D7FA0B349
:1001A00096FDA095A2FD5FEF451741F7A8E161FD1F
:1001B000A093680085FD03C0A8E1A0936800409368
:1001C0009700816085FD0EC0A0916900AA2331F0DF
:1001D000A0916900AA95A093690004C08061AA2734
:1001E000A064AABF80FF38C0A09197004A2F61FF8A
:1001F0008E7F85FD18C0403F08F040EFA42FA295E8
:10020000AF704A0F5091B800533069F0A695A6958B
:1002100050FD01C0A69552FD03C0A41B4A2F03C088
:100220004A0F08F44FEFA091A0004A1708F44A2F94
:1002300040936100A72FA67079F0A0916D00A6955C
:10024000A69556E0A50F50916100A50FA0936100FF
:1002500018F4AFEFA0936100A0916100A093630038
:1002600040916300A0919C004A1708F04A2F542E39
:10027000A091A200AA2309F422C0542F5A1B10F403
:10028000A42F50E0BA2E8894AA1FAA2EA091A400F1
:10029000A095AA22A50E58F0A091A300A21509F0DE
:1002A000AA95AA0EA093A30048F04A2D08C0A091D9
:1002B000A300BA1608F0A395A093A3004FEF4093B4
:1002C00064007F7D485F08F07062A52DA03408F0BF
:1002D0006860A0916000A395A093600051F0F8942D
:1002E000A9B7A160A9BF84FF02C0A0E4ABBF3FBE15
:1002F0001895A0917400A395A093740041E05091CB
:100300006800552329F085FF03C05A955093680073
:10031000A0919700A13018F020929A000DC0209271
:100320009B002092A500A0919A00AF5FA0939A0035
:1003300018F0AFEFA0939A00F894A9B7A160A9BFF5
:1003400084FF02C0A0E4ABBF3FBE18953FB64CB5DA
:100350005DB58F7EABB7A074A2118061A0E0ABBF8A
:10036000A9B7AE7FA9BF789481FD23C0A2E096FD16
:10037000A3E0A5BF8260A0B396FDA095A2FF05C033
:1003800040936500509366003EC1A3E096FDA2E055
:10039000A5BFAA27A064AABF8D7F85FF01C026C183
:1003A00040E0A0B396FDA095A2FD20C14093970028
:1003B0000FC1A3E096FDA2E0A5BF8D7F61FF71C0D4
:1003C000A2E096FDA3E0A5BFAA27A064AABF826011
:1003D0004093920050939300A09090004A19B090DF
:1003E00091005B09BB24A22C4C38520518F42092D2
:1003F000960049C0A091D600AA2359F1483C520565
:1004000028F4A0E1BA2EAAE0AA2E23C04836A1E023
:100410005A0728F4A8E0BA2EAFE0AA2E1AC0403D31
:10042000A2E05A0728F4A4E0BA2EAEE1AA2E11C029
:10043000403AA5E05A0728F4A2E0BA2EACE3AA2E6F
:1004400008C04839A8E05A0720F4A1E0BA2EA8E76E
:10045000AA2EC42EA0919400CA1AD52EA091950060
:10046000DA0ADD202AF4AFEFC094D094CA1ADA0A6F
:1004700020929600A8E0A210A0E0CA14DA0618F4B0
:10048000A1E0A09396004093940050939500409172
:10049000920050919300409390005093910002E09D
:1004A00097C0A09165004A1BA09166005A0B94FD6D
:1004B00082C093FD80C092FD7CC086FF03C0D52E14
:1004C000C42E0CC05695479591FD73C0569547951F
:1004D00090FD6FC0D52EC42ED694C79461FD19C06F
:1004E000AC2DAC51AD2DA24008F005C0DD2089F443
:1004F000AC2DA85C70F4A0916700A395AA2311F01D
:10050000A0936700AA3008F471C020929700816020
:100510006DC0A0916700AA2319F0AA95A093670067
:10052000A22C5091BC0097FD06C0A090CA00533089
:1005300011F4A090D200AAEFAA0EA22DA21DCA18F3
:10054000DA0A4FB74170533049F4442321F087FD54
:1005500005C0806803C087FF01C08F77442359F02E
:10056000533031F4AFEFC094D094CA1ADA0A03C002
:1005700040E050E020C0533049F4CC0CDD1CAAE030
:10058000CA1AD20818F4A0E0CA2ED22CAFEFCA16AD
:10059000D20418F04FEF50E00EC0A091AE00CA9EFA
:1005A000412D000C441F50E008F012C04FEF50E006
:1005B0000FC05695479594FF07C0552309F04FEF9C
:1005C000A42FA6954A0F521D4F3F520508F04FEF3A
:1005D00040939700816061FF09C0AFE1A095A92316
:1005E000AB299A2F8F7DBB2009F48062A8E1A093EC
:1005F000680085FF03C0AAE0A093680061FD03C006
:1006000085FD01C08F7E85FD03C0A6E0A093690033
:10061000F894A9B7A160A9BF84FF02C0A0E4ABBF52
:100620003FBE189511E00AC013E008C01AE006C0EA
:100630001EE104C014E602C018EC00C005E1BB27AF
:10064000BA95F1F70A95D9F71A95C1F708952AE3F3
:1006500038E709C020E33CE806C02AE234EB03C0D7
:1006600025E238EC00C012E095FD9F7D95FF906279
:10067000BB279498BA95F1F7C19ABA95F1F7C1984A
:10068000BA95F1F7949ABA95F1F7C09AB091AF0084
:10069000BA95F1F7C098B7E8BA95F1F71A9521F72E
:1006A000022FB22FBA95F1F70A95D9F73A95D9F6F4
:1006B00094980895221B39E0001F3A9509F4089593
:1006C000221F211B18F4210F8894F6CF0894F4CF31
:1006D000622C722CB0E08894B395221F331FE0F790
:1006E000379527958894912E802E020B130B10F4CA
:1006F000192D082D10F4889401C00894661C771CED
:10070000BA9571F7172D062D0895322D11232AF46D
:100710003A9500951095031B130BF894029F712CCA
:10072000002D129F912C802C7894780C172D921C00
:10073000292DB4E06B2E2695179507956A94D9F765
:10074000332321F000951095031B130B0895089592
:1007500010917B00169500917A000795B0917F006B
:10076000B01B0B2FB0918000B10B1B2F28F4003869
:10077000BFEF1B0740F009C00F37120508F405C092
:100780000FE710E002C000E81FEF00938400109311
:100790008500089500918400B09181000B0F1091A5
:1007A0008500B09182001B1F20E03091850033232B
:1007B0000AF42A95B09183002B1F1AF4203F40F0D1
:1007C0000AC02F3008F407C00FEF1FEF2FE003C05F
:1007D00000E010E020EF30916300B0919C003B17E7
:1007E00018F4323030F009C0B0918500BB235AF0C4
:1007F00004C0B0918500BB2332F4009381001093B4
:1008000082002093830008952091D80000918400F5
:10081000000F10918500111F78DF11232AF4003892
:10082000BFEF1B0740F009C00F37120508F405C0E1
:100830000FE710E002C000E81FEF002352F0B09174
:100840006200B01B0B2F18F0013008F00AC001E065
:1008500008C000950F5FB09162000B0F08F001C057
:100860000FEF0093860008952091D9000091820037
:10087000109183004ADF11232AF40130BFEF1B07D8
:1008800040F009C00F3F120508F405C00FEF10E05B
:1008900002C001E01FEF112352F0B0918600B01B9F
:1008A0000B2F18F0013008F00AC001E008C00095D5
:1008B0000F5FB09186000B0F08F001C00FEF00939F
:1008C000630008950FEF677F71FD29C072FD09C0B5
:1008D0006860B0917B00BA3020F0B52DB03408F4D8
:1008E000677FB091D500BB23D1F0B0917B00BB23D3
:1008F000B1F00FEF10917B00DDDEF894B091730042
:1009000072FDB5E00B9F112D002D7894112309F095
:100910000FEFB0919F000B1710F400919F00009310
:100920009E00089500917A0010917B0000541140C0
:10093000B0919E0010F4BA9501C0B39511F0B09338
:100940009E00089500C008952091B700B6B1B6FD8D
:10095000FBCF04B115B1B6B1BF77B6B9B091AC0059
:10096000B395B093AC00B83060F12092AC00B09178
:10097000D400BB2321F1112329F0B091AD00BF3F7A
:1009800061F009C0B091AD000B1739F020F4BB2322
:1009900021F0BA9502C0B395E1F300919C00B093A9
:1009A000AD00BA3F50F400ECB93F38F400E8B83F6E
:1009B00020F400E4B73F08F400E000939C00777F48
:1009C0000895B0919C00B39511F0B0939C00B09144
:1009D000AC00B73009F47860089502E3F894B09160
:1009E000DA000B9F012D000C001F7894B0919C0041
:1009F0000B1710F000919C000093610000936300BE
:100A0000502E0093640000939F00089520927A0076
:100A1000B0EFB0937B000895F8940CB51DB520910C
:100A200074007894309175006090760000937500A2
:100A300010937600031B160971FD03C076FD81C07B
:100A40002BC070907700209377002709222311F0A4
:100A50000FEF1FEF8090780090907900309378002E
:100A6000609279006918161910937C000091750046
:100A7000109176000819190920917A0030917B00B5
:100A800036952795020F131F10F40FEF1FEF0093F9
:100A90007A0010937B0029C020917A0030917B006E
:100AA0003901B4E08B2EB2E09B2E343010F08A94E2
:100AB0009A94383010F08A949A94769467948A9431
:100AC000E1F726193709992021F0169507959A9490
:100AD000E1F7200F311F20937A0030937B0028F438
:100AE0003FEF30937A0030937B00323008F470642B
:100AF00071FF02C0B3E00DC0B091C600009171005B
:100B0000023838F0B395003A08F0B395B63008F0E3
:100B1000B5E09B2EB4E08B2E10917B0000917A0003
:100B200024E0169507952A95E1F70819120928F08F
:100B3000B02FB250B12FB20910F402E010E09801CA
:100B400026C020917A0030917B0039017694679419
:100B50006694669466942619320906950695200FC8
:100B6000321D20937A0030937B00323008F07F7B77
:100B700004E0369527953695279526952695201BD2
:100B800010F0223008F422E089019090C60060FD48
:100B9000FECFE0908C00F0908D006160B9B7B0613D
:100BA000B9BF380176FD44C07694679400938C00F9
:100BB00010938D00B92DB330E1F0B0FD04C0060DE7
:100BC000171D930106C0000F111F0250120922E0E9
:100BD00030E0B92DB33068F020938E0030938F0051
:100BE000009388001093890060928A0070928B00B5
:100BF0003DC000938E0010938F00209388003093A7
:100C0000890060928A0070928B0071FF10C0B091D1
:100C10006D00B33060F000918F0010917C0015954D
:100C2000010F28F022F020928E0000938F001EC04A
:100C3000669400938C00B92DB33091F0B0FD03C0E1
:100C4000060D262D03C0000F025022E0B92DB3304F
:100C500038F020938E000093880060928A0006C0CE
:100C600000938E002093880060928A0000917D009E
:100C700002FD0350013031F495FD0FC0B0B7B77FCE
:100C8000B0BF11C0023039F4B0B7B860B0BFB4E043
:100C9000B06CB7B908C095FDF1CFB0B7B860B0BFC0
:100CA000B5E0B06CB7B90091A400000F10F4BBE63A
:100CB0000B270093A40060FDFECFB2E0B0936E005E
:100CC0006160B9B7B061B9BFB72FB670A1F020911C
:100CD0007A0030917B0036952795F8940CB51DB5B8
:100CE000020F131F1BBD0ABD6160B0E1B8BFB9B7E9
:100CF000B061B9BF78940895606120927E0020E0D1
:100D000067FD20E206C0606120927E0020E267FD60
:100D100020E0789401E076FD11C0B72FB67009F09D
:100D20006F7EB0917B00B55048F002E0B55020F0E6
:100D300003E0B55008F006E071FD0AE060FD12C066
:100D4000B0917E00BB2371F071FF08C0B0916D00BF
:100D5000B33020F0B0916E00BA9519F478947061B8
:100D60005EC0AEDF789400000000F89476FD16C0F7
:100D700010917B00173008F017E0B5E01B0F72FDF3
:100D800010E183FF110F62FF110F71FD12E8B4B57E
:100D90006090A100B61990F2B10B80F2B0B71B2F92
:100DA000B77FB0BFB8B1B0B713FDB860B0BFB091F6
:100DB0007E00B395B0937E00B8B176FD06C0B1E079
:100DC00071FDB2E0BA95F1F7B8B1B072B21709F09F
:100DD0001BC071FF05C003950A3008F00395AECF24
:100DE00064FF97CF6F7E3CB56DB470907A008090B1
:100DF0007B00370D681C6BBC3ABD6160B0E1B8BFC9
:100E0000B9B7B061B9BF85CFB0916D00B23008F409
:100E100080CF64FD7ECF0A9509F090CF7F7E209130
:100E20008E0030918F00F894B0E1B8BF0CB51DB5BD
:100E3000020F131F1BBD0ABDE0908800F0908900CF
:100E40006160B9B7B061B9BF7894B72FB67039F0A7
:100E5000B0916D0072FFB395B0936D0009C074FF3F
:100E600007C067FD05C064FD03C0BF91BF91E3C427
:100E7000089500E063FF03C064FF01C001E0F8943F
:100E800010917100B7E01B9F212D102D7894200F39
:100E90002695179526951795269517951093710009
:100EA000183718F4B8E7B093710000917100B09151
:100EB00072000B1720F06062C098C198C29860FD64
:100EC000FECFE0908A00F0908B006160B9B7B0610E
:100ED000B9BF0895B2E095FD07C0F894B0937D00C6
:100EE0009498939A7894E5C0F894B0937D00949880
:100EF000959A7894DEC0B3E082FF24C095FD11C0BE
:100F000002E0F894B0937D00E5E8F0E00093B300D0
:100F1000C298959862FF02C0C19A01C0949A7894D1
:100F2000C8C002E0F894B0937D00E5E8F0E00093DB
:100F3000B300C098939862FF02C0C19A01C0949A0E
:100F40007894B7C095FD0BC0F894B0937D00EFE6A0
:100F5000F0E0C29862FF01C0C19A7894AAC0F894E8
:100F6000B0937D00EFE6F0E0C09862FF01C0C19A47
:100F700078949FC0B4E095FD07C0F894B0937D00CD
:100F80009398959A789495C0F894B0937D0095982D
:100F9000939A78948EC0B5E082FF24C095FD11C06D
:100FA00001E0F894B0937D00EBE7F0E00093B3002C
:100FB000C198949862FF02C0C09A01C0939A789435
:100FC00078C004E0F894B0937D00EFE8F0E000937F
:100FD000B300C198949862FF02C0C29A01C0959A6A
:100FE000789467C095FD0BC0F894B0937D00E9E656
:100FF000F0E0C19862FF01C0C09A78945AC0F8949A
:10100000B0937D00E5E7F0E0C19862FF01C0C29AAD
:1010100078944FC0B6E095FD07C0F894B0937D007A
:101020009598949A789445C0F894B0937D009398DD
:10103000949A78943EC0B1E082FF24C095FD11C01F
:1010400004E0F894B0937D00EFE8F0E00093B30083
:10105000C098939862FF02C0C29A01C0959A789492
:1010600028C001E0F894B0937D00EBE7F0E0009336
:10107000B300C298959862FF02C0C09A01C0939ACB
:10108000789417C095FD0BC0F894B0937D00E5E708
:10109000F0E0C09862FF01C0C29A78940AC0F89448
:1010A000B0937D00E9E6F0E0C29862FF01C0C09A0B
:1010B00078946F7D089528E630E0F9012092B3001E
:1010C000C098C198C2989398949895986B7F08950A
:1010D000A4EBB0E00FEF0D930D930D930D9303E090
:1010E0000D9304E00D9309E00D9303E00D9301E0EF
:1010F0000D9301E00D93A0ECB0E001E00D930FEF34
:101100000D930D930D930D930D9303E00D930FEF3E
:101110000D930FEF0D930D9305E20D9300ED0D93DD
:101120000AEF0D930AEF0D9304E00D930FEF0D936B
:1011300001E00D9300E00D930AE70D930FEF0D937F
:1011400000E00D9301E00D9300E00D9303E00D939B
:1011500008952091BB008B7F233009F48460B09107
:10116000BC00B33019F09F7DB1FD90629F7BB091C0
:10117000BD00B1FD9064223011F0886001C0877F0E
:1011800008950A95E00FF21DB4910895ECE1F0E0A6
:101190000091B400F6DFB093D800ECE1F0E00091EC
:1011A000B500EFDFB093D900EAE2F0E00091BA00B9
:1011B000E8DFB093DA00B091D0000FEF1CE0B2305E
:1011C00011F400EA1AE0B33011F402E815E00093DC
:1011D000720010937300E8E3F0E00091D700D1DFD4
:1011E000B093A200089508952091CA003091CB00D9
:1011F000B091BC00B33009F43E5097FF02C020E02C
:101200003FEFB32FB21B6B2EB25810F4B2E86B2E27
:1012100000E00395609EB12DBD57D8F30093AE005A
:1012200008959068E1DF04DA20E030E0B0E16B2E51
:10123000FBD9B09197002B0F321D6A94C9F7B4E027
:1012400036952795BA95E1F7822E9F77CDDF0895E1
:10125000F894E3E0F0E0B9E0B7BFB491B078C1F33F
:10126000F894A895B1B5B861B1BDB0E0B1BDB4E036
:10127000BEBFBFE5BDBF1FDFB0E0B8BBB7E1B7BBC6
:10128000B0E0B5BBB0E0B4BBB0E0B2BBB8E3B1BB5B
:101290002224A0E0B0E02D92AA31E9F7A0E6B0E068
:1012A0000FEF2D920A95E9F7B1E0B093A40010DF9B
:1012B000F6D2B0E0B06CB7B9B6B1B460B068B6B948
:1012C0000091CC000093AF00B1E0B0936A00F894B5
:1012D000B3D9BDD9ADD9BED9ABD9BFD9A9D966D3F8
:1012E000ABD9AAD9A7D9F8940AEF1AEFA0B396FD03
:1012F000A095A2FF1FC01A95C9F70A95B1F7E0E0C3
:10130000FCE1B591B43E39F4B591B03E21F4B5910C
:10131000BF3F09F40CC0E0E0F395F395B591B83FF9
:1013200049F4B591B43931F4B591BA3A19F4EE27CC
:10133000F69509940EDF2ADF56DF56DF0091CC00C8
:101340000093AF00B8DEB2E0B3BFB2E0BEBDB2E022
:10135000B5BDB1E5B8BFB9BFB0B70B2FB77FB0BF50
:10136000B8B1B0B703FDB860B0BF5CD97894EADA21
:10137000B3E096FDB2E0B5BFB0E4BBBFBB27B0643D
:10138000BABF8D7F59D9626033E02CE0B0919600EE
:10139000BB2321F42CE03A9509F4A5CF49D980FF6D
:1013A000A2CF8E7FB0919700B23078F3B92FBF7182
:1013B0000091990000939800B0939900B01729F715
:1013C0002A9521F76D7FB3E096FDB2E0B5BFBB274C
:1013D000B064BABF8D7FB091D600BB2321F4806288
:1013E000B92FB0709B2F8F7B2092670023D985FF88
:1013F00005C0B0916700BA3008F0806415D902E0EA
:1014000085FF01C000E0B0919700B017B8F3F894E1
:101410001ED91DD91CD978940FD920928700B0917C
:10142000BC00B33009F474C0FFD8B091C000B13033
:1014300008F46EC0B0916A00B13008F469C085FD4F
:1014400018C0B0919700BF3F08F462C0F89408D963
:101450007894F0D8B0919700B130C0F7F894F7D8ED
:10146000E5D8F5D87894E6D8B0919700BF3FB0F3AF
:10147000CFC2B8E09B2E9068F894B6DE7894DAD8A4
:10148000F8949F77B1DE80909700B0919700BF37B6
:10149000789408F445C0C6D8F894E2D878949A9421
:1014A00051F7BFDEB82DB550B093CB00C5D8F89436
:1014B00023D281D27894BAE09B2E9068F89494DE7F
:1014C0007894B8D8F8949F778FDE80909700B09189
:1014D0009700BF37789478F7A5D8F894B8D8A6D8ED
:1014E000B6D878949A9449F79CDEB82DBB5FB09338
:1014F000CA00A2D8F89400D26DD278949BD8F89400
:1015000073DE7894B0919700BF3F08F498CF80C203
:1015100000919700B09187000B1710F0009387009F
:1015200089D801E0B091BC00B35009F405E0B09156
:101530009700B01708F073CFF89492D891D890D84C
:1015400078947AD820926A0020926B0020926C00E6
:10155000B0916B00B395B0936B00BF3F69F5B0914C
:101560006C00B395B0936C00B091CE0009E1BA95D0
:1015700059F002E3BA9541F00DE7BA9529F00AEF68
:10158000BA9511F020926C00B0916C00B017A0F0E9
:10159000B0916C00BA95B0936C00B4EBB0936B0053
:1015A000B091CD00B093AF00F8945AD87894B09130
:1015B000CC00B093AF003ED839D8B0916800BB23BF
:1015C00019F485FF01C08FCE01E085FD01C006E062
:1015D000B0919700B01708F4BBCFB091BC00B350E6
:1015E00009F028D8B0916800BB2309F47CCEF894A8
:1015F00062DD209261002092620020926300522CF2
:10160000209264002092A3007894B091B900BB0F9F
:10161000B093A00020927F00209280002092810051
:1016200020928200209283002092AC0060E070E063
:1016300020927100B8E0B093AC007860F3D7B0E0CE
:1016400073FDB1E0B06CB7B9B6B1B068B064B6B90B
:10165000B6B1B6FDFDCF04B115B1B6B1BF77B6B91D
:10166000112309F00FEF0093AD006ED9B8E0B093ED
:10167000AC0078608090BB00B2E0B093BB0069DD45
:101680008092BB00F894BFEFB0939C00A6D9B091B4
:101690006100B0939C00B0939D00B0939E0078943D
:1016A000B1E0B0936100B09363005B2EB09364002F
:1016B000B093A600B0919B00B093A500B091BC0080
:1016C000B33019F49F7D87FD906271607260209243
:1016D0006D00A0DCB0DC9AD99FD998D99DD996D954
:1016E00006C0F89436DD78942092AC00777F0BDB4F
:1016F0002ED8BFDBEFDB90D9FFDA66FD29D876FF65
:10170000E1D876FD0FD9B5DBF6DB86D9FCDA66FDCC
:1017100041D8AFDB2FDC80D9EFDA66FD75D8A9DBC5
:101720003ADC7AD9F0DA66FD9FD8A3DB73DC74D992
:10173000E3DAB0E073FDB1E0B06CB7B9B6B1B06850
:10174000B064B6B996DB77DC67D9FED871FF23C0E9
:1017500067FD21C0B0919F00B0939C00B0939D00A5
:10176000B0919B00B093A500B1E0B093A60018E142
:101770002CE0B0916D00B11740F07D7F7460209334
:101780006F00BFEFB0939C0006C0B0919700B130DE
:1017900008F0ADCF5AC072FF10C067FD0EC0B09107
:1017A0006F00BA9511F47B7F9CCFB0936F00B0911E
:1017B0009700B13008F09BCF48C020927000B091E4
:1017C0009A0002E8B01708F040C085FF04C0B0914D
:1017D0006800BB23D1F1B091BC00B33081F495FD1A
:1017E00003C087FD04C00BC087FF01C008C067FDB0
:1017F00006C06068B0919F00B0939C008DCF00EF51
:1018000067FF05C0B0919F00B0939C0000E2B091CB
:101810007B00B01708F46BCF67FF17C06F779F7D11
:1018200087FD90627460B2E1B0936F00B0919F0049
:10183000B0939C005CCFB0917000B395B0937000F2
:10184000B0919700BB2309F002C020927000F89479
:1018500032DC8090BB00B2E0B093BB007ADC8092B7
:10186000BB00209261002092620020926300522C03
:10187000209264002092A0007E7F7894D3D61BDC57
:10188000B0E0B06CB7B9B6B1B460B068B6B985FFB6
:1018900005C0B0917000B53008F025CD55CEEDE013
:1018A000F0E023D00A3509F01BC0EEE0F0E01DD0D7
:1018B000053A09F015C03AE0A4EBB0E0E3E0F0E04F
:1018C00014D00D9331963A95D9F738E1A0ECB0E0F9
:1018D000EFE0F0E00AD00D9331963A95D9F702C0C7
:1018E000F7DB0AD0E7E2F0E00895E199FECFEEBB26
:1018F000FFBBE09A0DB308951ED03AE0A4EBB0E030
:10190000E3E0F0E00D910FD031963A95D9F738E148
:10191000A0ECB0E0EFE0F0E00D9105D031963A9503
:10192000D9F712D00895E199FECF0DBBEEBBFFBBF6
:10193000E29AE19A0895EDE0F0E00FEFF4DFEEE0D7
:10194000F0E00FEFF0DF0895EDE0F0E00AE5EBDF07
:10195000EEE0F0E005EAE7DF08953091B000009195
:10196000B100313011F40093B800323011F400931B
:10197000B900333011F40093BA00343011F40093FD
:10198000C600353011F40093BB00363011F40093DB
:10199000D700373011F40093D000383011F40093A1
:1019A000BC00393011F40093BD00089525E044D601
:1019B0002A95E9F708954BD64DD64FD651D636D64F
:1019C00046D648D64AD64CD631D641D643D645D649
:1019D00047D6089545D641D63DD639D627D640D6E6
:1019E0003CD638D634D622D63BD637D633D62FD6A9
:1019F00008958090B0009090B10029D628D627D6BF
:101A000015D68A94D1F72CD611D69A94E1F7089579
:101A1000F894D1DF7894CADFC9DFB1E0B093B000A9
:101A2000B1E0B093B1002092B200F894E2DF789474
:101A3000B5E06B2E70909700FFD5B09197007B16A4
:101A4000C9F7B13018F0BF3F40F107C086DFF89406
:101A500053DFB1DFB8E0B1BDA9DF6A9459F7B091A7
:101A6000B200B395B093B200B33008F4DECF9EDF7E
:101A7000B091B100B395B093B100F894B091B000BB
:101A8000BA95EEE3F0E0EB0FF21D04917894039524
:101A9000B091B100B01708F4C6CF88DF87DFB091EE
:101AA000B000B395B093B000B091B000BA3008F474
:101AB000B7CF0EDBF89420DFB8E0B1BD77DFC8CB3D
:00000001FF
